BL51 BANKED LINKER/LOCATER V6.22                                                        10/31/2017  15:58:27  PAGE 1


BL51 BANKED LINKER/LOCATER V6.22, INVOKED BY:
D:\KEIL_V5\C51\BIN\BL51.EXE .\obj\main.obj, .\obj\sys.obj, .\obj\STARTUP.obj, .\obj\LCD.obj TO .\obj\ceshi PRINT (.\cesh
>> i.m51) RAMSIZE (256) DISABLEWARNING (16)


MEMORY MODEL: LARGE


INPUT MODULES INCLUDED:
  .\obj\main.obj (MAIN)
  .\obj\sys.obj (SYS)
  .\obj\STARTUP.obj (?C_STARTUP)
  .\obj\LCD.obj (LCD)
  D:\KEIL_V5\C51\LIB\C51L.LIB (?C_INIT)


LINK MAP OF MODULE:  .\obj\ceshi (MAIN)


            TYPE    BASE      LENGTH    RELOCATION   SEGMENT NAME
            -----------------------------------------------------

            * * * * * * *   D A T A   M E M O R Y   * * * * * * *
            REG     0000H     0008H     ABSOLUTE     "REG BANK 0"
            IDATA   0008H     0001H     UNIT         ?STACK

            * * * * * * *  X D A T A   M E M O R Y  * * * * * * *
            XDATA   0000H     0011H     UNIT         ?XD?LCD
            XDATA   0011H     000CH     UNIT         _XDATA_GROUP_

            * * * * * * *   C O D E   M E M O R Y   * * * * * * *
            CODE    0000H     0003H     ABSOLUTE     
            CODE    0003H     0285H     UNIT         ?PR?LCD_INIT?LCD
            CODE    0288H     008CH     UNIT         ?C_C51STARTUP
            CODE    0314H     0081H     UNIT         ?PR?_LCD_CLEAR?LCD
            CODE    0395H     007FH     UNIT         ?PR?_LCD_SETWINDOWS?LCD
            CODE    0414H     004AH     UNIT         ?PR?MAIN?MAIN
            CODE    045EH     0039H     UNIT         ?PR?LCD_SETPARAM?LCD
            CODE    0497H     002AH     UNIT         ?PR?_LCD_DRAWPOINT?LCD
            CODE    04C1H     0026H     UNIT         ?PR?_DELAY_MS?SYS
            CODE    04E7H     0026H     UNIT         ?PR?_DELAY_US?SYS
            CODE    050DH     001FH     UNIT         ?PR?_LCD_SETCURSOR?LCD
            CODE    052CH     001BH     UNIT         ?PR?LCD_RESET?LCD
            CODE    0547H     0017H     UNIT         ?PR?_LCD_WR_REG?LCD
            CODE    055EH     0017H     UNIT         ?PR?_LCD_WR_DATA?LCD
            CODE    0575H     0017H     UNIT         ?PR?_LCD_WR_DATA_16BIT?LCD
            CODE    058CH     0014H     UNIT         ?PR?_LCD_WRITEREG?LCD
            CODE    05A0H     000BH     UNIT         ?PR?LCD_WRITERAM_PREPARE?LCD
            CODE    05ABH     000BH     UNIT         ?C_INITSEG



OVERLAY MAP OF MODULE:   .\obj\ceshi (MAIN)


SEGMENT                                XDATA_GROUP
  +--> CALLED SEGMENT                START    LENGTH
----------------------------------------------------
BL51 BANKED LINKER/LOCATER V6.22                                                      10/31/2017  15:58:27  PAGE 2


?C_C51STARTUP                        -----    -----
  +--> ?PR?MAIN?MAIN
  +--> ?C_INITSEG

?PR?MAIN?MAIN                        -----    -----
  +--> ?PR?LCD_INIT?LCD
  +--> ?PR?_LCD_CLEAR?LCD
  +--> ?PR?_DELAY_MS?SYS

?PR?LCD_INIT?LCD                     -----    -----
  +--> ?PR?LCD_RESET?LCD
  +--> ?PR?_LCD_WRITEREG?LCD
  +--> ?PR?_DELAY_MS?SYS
  +--> ?PR?LCD_SETPARAM?LCD

?PR?LCD_RESET?LCD                    -----    -----
  +--> ?PR?_DELAY_MS?SYS

?PR?_LCD_WRITEREG?LCD                -----    -----
  +--> ?PR?_LCD_WR_REG?LCD
  +--> ?PR?_LCD_WR_DATA?LCD

?PR?LCD_SETPARAM?LCD                 -----    -----
  +--> ?PR?_LCD_WRITEREG?LCD

?PR?_LCD_CLEAR?LCD                   0011H    0004H
  +--> ?PR?_LCD_SETWINDOWS?LCD
  +--> ?PR?_LCD_WR_DATA_16BIT?LCD

?PR?_LCD_SETWINDOWS?LCD              0015H    0008H
  +--> ?PR?_LCD_WRITEREG?LCD
  +--> ?PR?LCD_WRITERAM_PREPARE?LCD

?PR?LCD_WRITERAM_PREPARE?LCD         -----    -----
  +--> ?PR?_LCD_WR_REG?LCD



SYMBOL TABLE OF MODULE:  .\obj\ceshi (MAIN)

  VALUE           TYPE          NAME
  ----------------------------------

  -------         MODULE        MAIN
  C:0000H         SYMBOL        _ICE_DUMMY_
  D:00B2H         PUBLIC        P3M0
  D:0090H         PUBLIC        P1
  D:00B1H         PUBLIC        P3M1
  D:00B0H         PUBLIC        P3
  C:0414H         PUBLIC        main
  -------         PROC          MAIN
  C:0414H         LINE#         52
  C:0414H         LINE#         53
  C:0414H         LINE#         57
  C:041AH         LINE#         60
  C:041DH         LINE#         63
  C:041DH         LINE#         64
BL51 BANKED LINKER/LOCATER V6.22                                                      10/31/2017  15:58:27  PAGE 3


  C:041DH         LINE#         65
  C:0432H         LINE#         66
  C:0447H         LINE#         67
  C:045CH         LINE#         68
  -------         ENDPROC       MAIN
  -------         ENDMOD        MAIN

  -------         MODULE        SYS
  C:0000H         SYMBOL        _ICE_DUMMY_
  C:04C1H         PUBLIC        _delay_ms
  C:04E7H         PUBLIC        _delay_us
  -------         PROC          _DELAY_MS
  D:0006H         SYMBOL        count
  -------         DO            
  D:0004H         SYMBOL        i
  D:0002H         SYMBOL        j
  -------         ENDDO         
  C:04C1H         LINE#         2
  C:04C1H         LINE#         3
  C:04C1H         LINE#         5
  C:04D1H         LINE#         6
  C:04E6H         LINE#         7
  -------         ENDPROC       _DELAY_MS
  -------         PROC          _DELAY_US
  D:0006H         SYMBOL        count
  -------         DO            
  D:0004H         SYMBOL        i
  D:0002H         SYMBOL        j
  -------         ENDDO         
  C:04E7H         LINE#         9
  C:04E7H         LINE#         10
  C:04E7H         LINE#         12
  C:04F7H         LINE#         13
  C:050CH         LINE#         14
  -------         ENDPROC       _DELAY_US
  -------         ENDMOD        SYS

  -------         MODULE        ?C_STARTUP
  C:0288H         SEGMENT       ?C_C51STARTUP
  I:0008H         SEGMENT       ?STACK
  C:0000H         PUBLIC        ?C_STARTUP
  D:00E0H         SYMBOL        ACC
  D:00F0H         SYMBOL        B
  D:0083H         SYMBOL        DPH
  D:0082H         SYMBOL        DPL
  N:0000H         SYMBOL        IBPSTACK
  N:0100H         SYMBOL        IBPSTACKTOP
  N:0080H         SYMBOL        IDATALEN
  C:028BH         SYMBOL        IDATALOOP
  N:0000H         SYMBOL        PBPSTACK
  N:0100H         SYMBOL        PBPSTACKTOP
  N:0000H         SYMBOL        PDATALEN
  N:0000H         SYMBOL        PDATASTART
  N:0000H         SYMBOL        PPAGE
  N:0000H         SYMBOL        PPAGEENABLE
  D:00A0H         SYMBOL        PPAGE_SFR
  D:0081H         SYMBOL        SP
BL51 BANKED LINKER/LOCATER V6.22                                                      10/31/2017  15:58:27  PAGE 4


  C:0288H         SYMBOL        STARTUP1
  N:0000H         SYMBOL        XBPSTACK
  N:0000H         SYMBOL        XBPSTACKTOP
  N:0000H         SYMBOL        XDATALEN
  N:0000H         SYMBOL        XDATASTART
  C:0000H         LINE#         126
  C:0288H         LINE#         133
  C:028AH         LINE#         134
  C:028BH         LINE#         135
  C:028CH         LINE#         136
  C:028EH         LINE#         185
  C:0291H         LINE#         196
  -------         ENDMOD        ?C_STARTUP

  -------         MODULE        LCD
  C:0000H         SYMBOL        _ICE_DUMMY_
  D:0080H         PUBLIC        P0
  D:0090H         PUBLIC        P1
  D:00A0H         PUBLIC        P2
  D:00B0H         PUBLIC        P3
  C:0547H         PUBLIC        _LCD_WR_REG
  C:0314H         PUBLIC        _LCD_Clear
  B:00B0H.3       PUBLIC        LCD_RESET
  C:052CH         PUBLIC        LCD_Reset
  C:0575H         PUBLIC        _LCD_WR_DATA_16Bit
  B:00B0H.2       PUBLIC        LCD_BL
  C:0003H         PUBLIC        LCD_Init
  B:0090H.3       PUBLIC        LCD_CS
  B:0090H.0       PUBLIC        LCD_RD
  C:0497H         PUBLIC        _LCD_DrawPoint
  C:0395H         PUBLIC        _LCD_SetWindows
  C:045EH         PUBLIC        LCD_SetParam
  C:05A0H         PUBLIC        LCD_WriteRAM_Prepare
  C:055EH         PUBLIC        _LCD_WR_DATA
  B:0090H.2       PUBLIC        LCD_RS
  B:0090H.1       PUBLIC        LCD_WR
  C:0592H         PUBLIC        _LCD_WriteReg
  C:050DH         PUBLIC        _LCD_SetCursor
  X:0000H         PUBLIC        POINT_COLOR
  X:0002H         PUBLIC        BACK_COLOR
  X:0004H         PUBLIC        lcddev
  -------         PROC          _LCD_WR_REG
  D:0004H         SYMBOL        Reg
  C:0547H         LINE#         62
  C:054BH         LINE#         63
  C:054BH         LINE#         64
  C:054DH         LINE#         65
  C:054FH         LINE#         69
  C:0553H         LINE#         70
  C:0557H         LINE#         72
  C:0559H         LINE#         73
  C:055BH         LINE#         74
  C:055DH         LINE#         75
  -------         ENDPROC       _LCD_WR_REG
  -------         PROC          _LCD_WR_DATA
  D:0004H         SYMBOL        Data
  C:055EH         LINE#         86
BL51 BANKED LINKER/LOCATER V6.22                                                      10/31/2017  15:58:27  PAGE 5


  C:0562H         LINE#         87
  C:0562H         LINE#         88
  C:0564H         LINE#         89
  C:0566H         LINE#         93
  C:056AH         LINE#         94
  C:056EH         LINE#         96
  C:0570H         LINE#         97
  C:0572H         LINE#         98
  C:0574H         LINE#         99
  -------         ENDPROC       _LCD_WR_DATA
  -------         PROC          _LCD_WR_DATA_16BIT
  D:0004H         SYMBOL        Data
  C:0575H         LINE#         110
  C:0579H         LINE#         111
  C:0579H         LINE#         112
  C:057BH         LINE#         113
  C:057DH         LINE#         122
  C:0581H         LINE#         123
  C:0585H         LINE#         124
  C:0587H         LINE#         125
  C:0589H         LINE#         127
  C:058BH         LINE#         128
  -------         ENDPROC       _LCD_WR_DATA_16BIT
  -------         PROC          L?0021
  -------         ENDPROC       L?0021
  -------         PROC          _LCD_WRITEREG
  D:0006H         SYMBOL        LCD_Reg
  D:0002H         SYMBOL        LCD_RegValue
  C:0592H         LINE#         140
  C:0596H         LINE#         141
  C:0596H         LINE#         142
  C:0599H         LINE#         143
  -------         ENDPROC       _LCD_WRITEREG
  -------         PROC          LCD_WRITERAM_PREPARE
  C:05A0H         LINE#         156
  C:05A0H         LINE#         157
  C:05A0H         LINE#         158
  -------         ENDPROC       LCD_WRITERAM_PREPARE
  -------         PROC          _LCD_CLEAR
  X:0011H         SYMBOL        Color
  -------         DO            
  X:0013H         SYMBOL        i
  D:0002H         SYMBOL        j
  -------         ENDDO         
  C:0314H         LINE#         171
  C:031CH         LINE#         172
  C:031CH         LINE#         174
  C:0346H         LINE#         175
  C:0362H         LINE#         176
  C:0362H         LINE#         177
  C:0372H         LINE#         178
  C:0372H         LINE#         179
  C:037DH         LINE#         180
  C:0384H         LINE#         182
  C:0394H         LINE#         183
  -------         ENDPROC       _LCD_CLEAR
  -------         PROC          _LCD_DRAWPOINT
BL51 BANKED LINKER/LOCATER V6.22                                                      10/31/2017  15:58:27  PAGE 6


  D:0002H         SYMBOL        x
  D:0082H         SYMBOL        y
  C:0497H         LINE#         194
  C:049FH         LINE#         195
  C:049FH         LINE#         196
  C:04B6H         LINE#         197
  -------         ENDPROC       _LCD_DRAWPOINT
  -------         PROC          LCD_RESET
  C:052CH         LINE#         209
  C:052CH         LINE#         210
  C:052CH         LINE#         211
  C:052EH         LINE#         212
  C:0535H         LINE#         213
  C:0537H         LINE#         214
  C:053EH         LINE#         215
  C:0540H         LINE#         216
  -------         ENDPROC       LCD_RESET
  -------         PROC          LCD_INIT
  C:0003H         LINE#         228
  C:0003H         LINE#         229
  C:0003H         LINE#         230
  C:0006H         LINE#         231
  C:0008H         LINE#         235
  C:0013H         LINE#         236
  C:001EH         LINE#         237
  C:0029H         LINE#         238
  C:0032H         LINE#         239
  C:0037H         LINE#         240
  C:0042H         LINE#         241
  C:0047H         LINE#         242
  C:0052H         LINE#         243
  C:005DH         LINE#         244
  C:0066H         LINE#         245
  C:006FH         LINE#         246
  C:007AH         LINE#         247
  C:0085H         LINE#         248
  C:0090H         LINE#         249
  C:009BH         LINE#         250
  C:00A6H         LINE#         252
  C:00AFH         LINE#         253
  C:00B8H         LINE#         254
  C:00C1H         LINE#         255
  C:00CCH         LINE#         256
  C:00D7H         LINE#         257
  C:00E2H         LINE#         258
  C:00EDH         LINE#         259
  C:00F6H         LINE#         260
  C:0101H         LINE#         261
  C:010CH         LINE#         262
  C:0117H         LINE#         263
  C:0122H         LINE#         264
  C:012BH         LINE#         265
  C:0136H         LINE#         266
  C:0141H         LINE#         267
  C:014CH         LINE#         268
  C:0157H         LINE#         269
  C:0162H         LINE#         270
BL51 BANKED LINKER/LOCATER V6.22                                                      10/31/2017  15:58:27  PAGE 7


  C:016DH         LINE#         271
  C:0178H         LINE#         272
  C:0183H         LINE#         273
  C:018EH         LINE#         274
  C:0199H         LINE#         275
  C:01A4H         LINE#         276
  C:01AFH         LINE#         277
  C:01BAH         LINE#         279
  C:01C5H         LINE#         280
  C:01D0H         LINE#         281
  C:01DBH         LINE#         282
  C:01E6H         LINE#         285
  C:01F1H         LINE#         287
  C:01FCH         LINE#         288
  C:0207H         LINE#         289
  C:0212H         LINE#         290
  C:0219H         LINE#         291
  C:0224H         LINE#         292
  C:022BH         LINE#         293
  C:0236H         LINE#         294
  C:023DH         LINE#         295
  C:0248H         LINE#         296
  C:024FH         LINE#         298
  C:025AH         LINE#         300
  C:0265H         LINE#         302
  C:0270H         LINE#         303
  C:0277H         LINE#         304
  C:0282H         LINE#         307
  C:0285H         LINE#         308
  C:0287H         LINE#         309
  -------         ENDPROC       LCD_INIT
  -------         PROC          _LCD_SETWINDOWS
  X:0015H         SYMBOL        xStar
  X:0017H         SYMBOL        yStar
  X:0019H         SYMBOL        xEnd
  X:001BH         SYMBOL        yEnd
  C:0395H         LINE#         316
  C:03A9H         LINE#         317
  C:03A9H         LINE#         319
  C:03B7H         LINE#         320
  C:03C3H         LINE#         321
  C:03D1H         LINE#         322
  C:03DDH         LINE#         323
  C:03EBH         LINE#         324
  C:03F7H         LINE#         325
  C:0405H         LINE#         326
  C:0411H         LINE#         328
  -------         ENDPROC       _LCD_SETWINDOWS
  -------         PROC          _LCD_SETCURSOR
  D:0002H         SYMBOL        Xpos
  D:0082H         SYMBOL        Ypos
  C:050DH         LINE#         337
  C:0515H         LINE#         338
  C:0515H         LINE#         339
  -------         ENDPROC       _LCD_SETCURSOR
  -------         PROC          LCD_SETPARAM
  C:045EH         LINE#         344
BL51 BANKED LINKER/LOCATER V6.22                                                      10/31/2017  15:58:27  PAGE 8


  C:045EH         LINE#         345
  C:045EH         LINE#         346
  C:0467H         LINE#         348
  C:046DH         LINE#         349
  C:0475H         LINE#         350
  C:047CH         LINE#         351
  C:0485H         LINE#         352
  C:048CH         LINE#         353
  -------         ENDPROC       LCD_SETPARAM
  -------         ENDMOD        LCD

Program Size: data=9.0 xdata=29 code=1462
LINK/LOCATE RUN COMPLETE.  0 WARNING(S),  0 ERROR(S)
